:020000040000FA
:10000000000083169F141F15003087008800FF3002
:10001000860081138312FF30870088000030A00023
:10002000A100A200A3003030900021281010AF30B2
:100030008E003C308F0010140C1C1C280C1010106B
:100040000800FE308800061C2014061D21146B20B9
:100050001620FD308800861CA014861EA114061FE1
:10006000A2146B201620FB308800061D2015061CEC
:100070002115861E22156B201620F7308800861D5C
:10008000A015861DA115061EA2156B201620EF30A7
:100090008800061E2016061E2116861D22166B20BD
:1000A0001620DF308800861EA016861CA116061DAD
:1000B000A2166B201620BF308800061F2017061FCF
:1000C0002117861C22176B2016207F308800861F80
:1000D000A017861FA117BF30061CF930861CA4305C
:1000E000061DB030861D9930061E9230861E823065
:1000F000061FF830861F80308700881B080088178D
:1001000016208630A300031118302002A4300319F2
:10011000A30003113C30200299300319A3000311FE
:100120007E30200282300319A3000311FF30200229
:100130008C300319A3000311FF302102C6300319CC
:10014000A30003117E30220282300319A3000311A1
:100150003C30220299300319A30003111830220207
:10016000A4300319A30016201620FF3087001620A4
:0801700023088700B4280000F9
:02400E00723FFF
:00000001FF
